:101C000000060020E17800006D6600006D660000AF
:101C100000000000000000000000000000000000C4
:101C20000000000000000000000000006D660000E1
:101C300000000000000000006D6600007120000040
:101C40000000000000000000000000000000000094
:101C5000000000006D6600006D6600006D6600000B
:101C6000F5530000000000006D6600000000000059
:101C7000E120000000000000000000006D66000090
:101C80006D6600006D6600006D66000000000000DB
:101C90006D6600006D66000000000000000000009E
:101CA0000000000000000000000000000000000034
:101CB0006D660000000000006D6600006D660000AB
:1020100010B5064C2378002B07D1054B002B02D0BE
:10202000044800E000BF0123237010BDB8FEFF1F6D
:10203000000000006C7B0000084B10B5002B03D0A3
:102040000749084800E000BF07480368002B00D19B
:1020500010BD064B002BFBD09847F9E700000000AD
:10206000BCFEFF1F6C7B0000B8FEFF1F00000000DD
:102070000E4A1368013313600D4A1368013313606D
:102080000C4B1A68002A08D01A68013A1A601B68BB
:10209000002B02D10122084B1A70084B1A68002A43
:1020A00002D01A68013A1A607047C046D4FEFF1F7A
:1020B00038030020F4020020F0020020F802002083
:1020C000024B034A5A6007221A60704710E000E092
:1020D00080BB0000014B18687047C046D4FEFF1F4C
:1020E000234B30B55868820214D5224A1168013159
:1020F000202900D100215468A14205D01468DD6870
:102100001419EDB22572116005241B490C60916A07
:102110001A4A1160420206D50421194A91609A6850
:1021200018490A409A6002021CD5144A1068002817
:1021300018D1104AD46A116B8C4214D0042410496F
:102140004C60116B4C1C146314003434615CC9B2D4
:10215000D960116B202900D1106380229968D203C5
:102160000A439A6030BD9A6807490A40F9E7C046B9
:1021700000400540D8FEFF1FF4020020F8020020B6
:1021800040F00F40FFFFBFFFFFFF7FFF0021144B18
:10219000144A70B599508022134C52031D592A439A
:1021A0001A518022114BD200DA601A61082800D936
:1021B00008000F4B8000C15811230E48594304F00A
:1021C0003BFB8023B022C0045B05C00C18430A4BC4
:1021D000920318609A600C2004F058FA70BDC04653
:1021E00000700440101000003810000000900440FF
:1021F00090790000006CDC02004005400A4A10B5EE
:10220000D36A0133202B00D10023116B8B420AD0FB
:102210001400D16A34346054D3628023034A1B040F
:1022200091680B43936010BDD8FEFF1F004005402E
:102230000A4B10B55C68196800228C420BD05A68B2
:10224000511C59609A18127A59680270012220298B
:1022500001D100215960100010BDC046D8FEFF1FFB
:10226000014B98627047C046D8FEFF1F0020034B09
:102270001A78824201D0187001307047F0020020B5
:10228000BFF34F8F024A034BDA60BFF34F8FFEE775
:102290000400FA0500ED00E0C0232C492C4ADB00C5
:1022A0008858F0B503438B5080212420294A2A4BBB
:1022B000490051615861043858602848222541601E
:1022C000816041612620264C85B060612238A06083
:1022D0006560116091600021009003380C000E00D1
:1022E0008446204F183D0192009898600396039809
:1022F000B84221D962461869104042424241A418AE
:10230000009A5A6003960398B84219D96246186930
:10231000013D10400918002DE6D1134B0A2C13D1B2
:102320000A2911D109391970C023019A9B00136041
:10233000019A936005B0F0BD039801300390D6E791
:10234000039801300390DEE70021ECE700700440C1
:10235000381000000090044000F00F4000A004403E
:1023600040F00F40E7030000B003002070477047C3
:1023700010B5002802D104F0BDF810BD0020FCE724
:1023800000207047704770470020704713B50D4B11
:102390001B78002B15D0022100200B4A0B4C9160BA
:1023A0000190019BA34208D951600190019BA34277
:1023B000F5D8019B01330193F8E7019B01330193A9
:1023C000EFE713BDB003002040F00F403F0D0300C6
:1023D00037B5092501AC210001226C20257003F0DE
:1023E000A5F8210002226C2003F0C6F80F23227802
:1023F000210013436C2002226370257003F096F8CD
:1024000000223821100003F0E7FBC8223A215203D2
:10241000002003F0E1FB00223921100003F0DCFB77
:1024200037BD0E2313B501AC210001226C202370AF
:1024300003F07CF8022221006C2003F09DF8208834
:1024400040BA80B216BDC04673B5B84CA578002D11
:1024500000D040E362788C2A00D1E8E200D9CFE0D6
:10246000122A00D132E269D8072A00D1D1E130D84E
:10247000022A00D17BE107D8002A00D15CE1012AC1
:1024800000D168E1032227E3052A00D199E100D9B0
:10249000ADE1042AF6D12379E0781B020343607989
:1024A000A34D00040343A07900061843C317C018C6
:1024B00058402B6898476860A078202103F0C2FB41
:1024C000002800D046E1A07827218300ED186A6833
:1024D0003EE10E2A00D1C4E11BD80C2A00D1A9E1AB
:1024E0000D2ACFD13421002003F0ACFB2179E37811
:1024F00009021943637902001B041943A379A078E8
:102500001B060B430121002B00D041E20A4333316B
:102510001EE18749102A00D1C9E100D8B8E123792A
:10252000E0781B020343607900040343A0790006AE
:1025300018438B6898472821020008E1192A00D126
:1025400010E234D8152A00D1E0E114D8132A00D1C2
:10255000CCE1142A96D12379E0781B0203436079F9
:1025600000040343A07900061843714B1B68984789
:102570002B210200EBE0172A00D1E3E100D8D1E1E2
:102580003421002003F05EFB2179E378090219432E
:10259000637902001B041943A379A0781B060B433F
:1025A0000821002B00D1F3E10A432C31D0E01F2A8F
:1025B00000D10DE20CD81B2A00D104E200D2EAE1DE
:1025C0001C2A00D05EE7E178002003F02BFCC1E07C
:1025D000212A00D11DE200D20BE27F2A00D051E770
:1025E0002279E178637912021B040A431A43A37922
:1025F0001B061343012B00D96DE24D4B1973A9E063
:10260000B62A00D1DCE23FD8A82A00D1BAE218D815
:10261000A42A00D17CE20AD8A22A00D173E2A32A1C
:1026200000D02FE7E178002003F012FC92E0A62A08
:1026300000D199E200D870E2E178002003F06AFB53
:1026400088E0AC2A00D1ACE209D8AA2A00D1A3E2E2
:1026500000D89CE2E178002003F0F1FC7AE0AE2A99
:1026600000D1A8E200D2A1E2B52A00D00AE722797F
:10267000E37812021A4363791B041A43A3791B06F9
:1026800013432C4A136165E0C02A00D1EEE11BD848
:10269000BA2A00D1B8E20AD8B82A00D1AFE2B92AE2
:1026A00000D0EFE6E178002003F068FB52E0BC2A9E
:1026B00000D1E4E200D2C6E2BF2A00D0E2E6E1782F
:1026C000002003F0BBFD45E0CC2A00D1DCE217D8A6
:1026D000C22A00D1D3E100D2CDE1C32A00D0D1E695
:1026E0002379E0781B020343607900040343A07957
:1026F000000618430E4B1B6898470E4B586029E0A4
:10270000D62A00D1CBE1FF2A00D1D7E1D12A00D0CF
:10271000B8E62379E2781B02134362793921120467
:102720001343A27912061A4311E0C046FC020020AE
:102730002CFFFF1FB40300202D212379E2781B0218
:102740001343627912041343A27912061A4300203C
:1027500003F042FA73BD2379E2781B0213436279D6
:10276000212112041343A27912061A43EFE72179BB
:10277000E3780902194363791B041943A3791B0603
:102780000B43002B00DD01222021280003F024FA56
:102790000122A578E64BE0785A552379AA001B025E
:1027A0000343607900040343A07900061843C3176C
:1027B000C0185840DF4BD358984727210200280003
:1027C000C6E70022DC4BE0781A7023791B02034332
:1027D000607900040343A07900061843D54B9B6839
:1027E0009847D64B02001860A0782621B0E7102148
:1027F000002003F027FA0200D2B2030CA078019265
:10280000E2781021D20800920022DBB203F098F99E
:10281000A0E71021280003F015FAE278A678030C4F
:10282000D208000A0192C2B20092DBB22A00102143
:102830003000EBE73421002003F004FA2179E3783B
:1028400009021943637902001B041943A379A07894
:102850001B060B430221002B00D099E00A433231C2
:1028600076E73421280003F0EDF92179E3780902B5
:102870001943637902001B041943A379A0781B064E
:102880000B431021002B00D182E00A4324315FE783
:102890002379E0781B020343607900040343A079A5
:1028A000000618438B689847242102004FE72379DC
:1028B000E0781B020343607900040343A07900061B
:1028C00018430B6898472521020040E72379E078F8
:1028D0001B020343607900040343A07900061843F8
:1028E000944B9B6898472A21020030E72379E078CF
:1028F0001B020343607900040343A07900061843D8
:102900008C4B1B6898472321020020E72379E2784B
:102910001B02134362792C2112041343A27912067D
:102920001A4314E72379E0781B020343607900041B
:102930000343A079000618437E4B1B689847152176
:10294000020004E72379E0781B0203436079000466
:102950000343A07900061843764B1B689847332140
:102960000200F4E63421280003F06CF92179E378C1
:1029700009021943637902001B041943A379A07863
:102980001B060B430421002B02D00A433031DFE643
:102990008A433421DCE63421002003F053F9217905
:1029A000E37809021943637902001B041943A379F0
:1029B000A0781B060B4303D080231B011A43E8E7D2
:1029C0005F4B1A40E5E7E178002003F015FAC1E615
:1029D0001021280003F036F90F22E378A478134081
:1029E000C2B2000A0192C2B2009210212A00200055
:1029F0000CE76E21002003F025F90321E278000C9A
:102A0000C3B2A078019222790A4000926B31002271
:102A1000FCE66E21002003F015F9C2B2000AE3784B
:102A2000A4780192C2B200926E210022DFE7082151
:102A3000E3782800C91AC9B203F0B4F92279E3781F
:102A400012021A436379A0781B041A43A3793A212E
:102A50001B061343802252029A401300D2175205DC
:102A6000520DD218C823D2125A4371E6E1782800D9
:102A700003F0CEFB6EE6E278324B1A726AE62379F7
:102A8000E0781B020343607900040343A079000649
:102A90001843284B1B6898472A4B18605AE623793D
:102AA000E2781B0213436279112112041343A279C5
:102AB00012061A43D30F9A18521048E62279E37887
:102AC00012021A4363791B041A43A3791B061343AA
:102AD00005D0012B0CD004221B4B1A703AE6194A80
:102AE0001376144B194A1A601A619A605A6131E6DA
:102AF000144A13760F4B164A1A60164A1A61164A80
:102B00009A60164AF2E7E178002003F023F921E603
:102B1000E178280003F0C8F91CE6002003F05CFA15
:102B2000E17800281CD1A07803F004FA12E6C04630
:102B3000A90300202CFFFF1F3404002030040020D4
:102B4000FFF7FFFFB40300203C0300209565000061
:102B50000D6500003D650000256500007D650000F5
:102B6000A07803F0B7F9F5E5002003F035FAE17835
:102B7000002803D1A07803F0DDF8EBE5A07803F09E
:102B8000C5F9E7E5E178280003F0B4FAE2E5E17879
:102B9000002003F064FADDE5E178002003F074FA28
:102BA000D8E5E178280003F083FAD3E5E178002046
:102BB00003F0B6FACEE5E178002003F089FAC9E522
:102BC0002179E07809020143607900040143A0798A
:102BD0000006084300D57EE72E4B1B7E012B01D05B
:102BE00003F0ACFC002807D001002B4803F024FEC2
:102BF0000200A0781421ABE5A078284AFAE7E17832
:102C0000002003F03BF9A5E52179E07809020143B2
:102C1000607900040143A0790006084300D55AE713
:102C20001C4B1B7E012B01D003F088FC002807D031
:102C30000100194803F000FE0200A078132187E587
:102C4000A078164AFAE7E178002003F00BFB002198
:102C5000A07802F0F7FF2379E1781B020B4361793A
:102C6000020009040B43A179A07809061943042343
:102C7000002902D01A4300216AE59A4368E5E17809
:102C8000002003F001FB65E5E178280003F096FAE7
:102C900060E5C046B40300200024F400B500100035
:102CA00070B5B24CA078022800D1D8E0032800D13A
:102CB000E4E0002800D057E16378512B00D184E094
:102CC0001CD8442B51D007D8412B40D0422B47D0A1
:102CD0000322A74B1A7042E04C2B56D04D2B62D0EA
:102CE0004B2BF5D1A34DE3780122A3490320EB70D0
:102CF00002F0F3F8E878FFF7B3FA30E0832B00D165
:102D000086E019D8552B00D16FE0572B44D0542BB7
:102D1000DED12279E178637912021B040A431A4357
:102D2000A3791B061343012B00D91DE1914B01220E
:102D300099730E20914910E0852B00D182E000D2DA
:102D400073E0FF2BC4D1E2788D4B1A7607E0E2786E
:102D5000884B02209A7001228A4902F0BEF870BDA9
:102D60008449E37801220B70F7E72279E3781202B5
:102D70001A43637984491B041A43A37908201B066C
:102D800013437C4A93600422E7E7E278794B7F495A
:102D90005A7001221000E0E7E278764B7C491A7104
:102DA00004200122D9E72279E37812021A436379D9
:102DB0001B041A43A3791B061343012BCFD86D4A7A
:102DC000744913730C200122C7E70123694D6A7B04
:102DD0001A4204D0E2781A4201D102F0D7F8E17821
:102DE0000D20697302F06BF8B9E72279E178637915
:102DF00012021B040A431A43A3791B061343012B37
:102E000000D9B1E05B4B0122D9730F206249A4E7DE
:102E10002279E37812021A4363791B041A43A379D7
:102E20001B061343564AD36199E72279E3781202CD
:102E30001A4363791B041A43A3791B061343574AA9
:102E400013608CE72279E37812021A4363791B043A
:102E50001A43A3791B061343494A13627FE7227979
:102E6000E37812021A43637961781B041A43A37949
:102E700089001B0613434A4A8B5070E76378272B5F
:102E80005FD020D8022B43D015D8002B2FD0012B98
:102E900000D01DE72279E37812021A4363791B04FC
:102EA0001A43A3791B0613433E4A5360FFF712F9F6
:102EB000334B986253E71B2B3BD01C2B3DD0092B87
:102EC00000D005E74BE72B2B43D006D8E2783549F5
:102ED000292B3CD039D94A7541E72D2B41D03CD321
:102EE0002E2B00D0F4E6E2782E4B5A7637E7227983
:102EF000E37812021A4363791B041A43A3791B0671
:102F00001343284A1360FFF7E5F81D4B586226E784
:102F10002279E37812021A4363791B041A43A379D6
:102F20001B0613431F4A9360FFF7D4F8144BD86273
:102F300015E7E2781B4B1A7411E7E278194B5A74C3
:102F40000DE7E278174B9A7409E7CA7407E70A7528
:102F500005E7E278134B9A7501E7E278114BDA75D1
:102F6000FDE6E2780F4BF0E60422B2E6FC02002018
:102F70003C0300200CFEFF1F0FFEFF1F1AFEFF1F69
:102F80002CFFFF1F0EFEFF1F14FEFF1F0DFEFF1F75
:102F900010FEFF1F18FEFF1F1BFEFF1F380300203F
:102FA00048030020D80300203649F8B50A00364B04
:102FB00031CB31C231CB31C211CB11C20B7E334C7C
:102FC000002B36D1324B23602361A36027210020E0
:102FD0000025636102F036FE2E4B6060262128003A
:102FE0001D7002F02FFE2C4B2A0018602B4B2C4F2B
:102FF0001D70230030331D702A4B65631D602A4B02
:103000001D602A4B1D60230038331D70EB190435F9
:103010001A60502DFAD1264EB37B002B11D1F37BD1
:10302000002B1ED0337B002B2AD001233934237090
:10303000F8BD204B2360204B2361204BA360204B25
:10304000C4E7D825AD001F4B2800E9181E4B042209
:10305000C91801F078FFE12304359B009D42F2D1AD
:10306000DDE7A025AD00194B2800E91879180422E6
:1030700001F069FFB42304359B009D42F3D1D1E7F1
:103080003934D4E7B4030020C07900002CFFFF1FBF
:1030900095650000A90300203004002034040020BE
:1030A00048030020300300204403002004030020D4
:1030B0000CFEFF1F0D6500003D650000256500004A
:1030C0007D650000A4FCFFFF0803002080FDFFFFDA
:1030D000F0B5C54E89B0337E002B04D133003A33AE
:1030E0001B78002B0DD0FB22C04B1B78991F11427F
:1030F00007D0EB3A93430F2B03D033000022303339
:103100001A70330030331B78012B00D024E13300D8
:103110003B331B78002B2CD1B54FB64D78783C78DB
:103120002B780419E4186B78E418EB79E418AB7980
:10313000E4186B79E4182B79E418FFF75FF8387816
:10314000FFF75CF82878FFF759F86878FFF756F82A
:10315000E879FFF753F8A879FFF750F86879FFF797
:103160004DF8E4B22879FFF749F82000FFF746F858
:103170000AE0012B08D1002433003C33E05C013429
:10318000FFF73CF8092CF7D19B4B1B78002B2AD07A
:103190009A4B9B4D1B78012B21D1954F2B7878783A
:1031A0003C7804190A34E418FFF728F83878FFF758
:1031B00025F88020FFF722F88A20FFF71FF800206B
:1031C000FFF71CF80020FFF719F80020FFF716F8AA
:1031D000E4B22878FFF712F82000FFF70FF8002379
:1031E000854A2B7013703200002330321370320086
:1031F0003B321370330045331B78002B04D0202260
:10320000804B5A60FFF73CF80F2402ABE418200013
:10321000FFF70EF8002800D1CBE0FFF727F80028D1
:1032200003D03300002246331A7032003100463298
:1032300010782478431CDBB2473113700C54092BEF
:1032400045D1002313706A4B0A781978914202D055
:10325000197991423BD11B7931009B1A5842584150
:103260003A310870002133000A004733C85C01314D
:103270001218D2B20829F9D13400197A30349142A7
:1032800000D093E05978594A117099785170D978E3
:103290009170197991715979517199791171DB791D
:1032A000D370FEF717FF584B584A1860002313706D
:1032B0003200463213703200012139321078217009
:1032C000441E534A8C426FD905286DD011703200CC
:1032D00039321178042906D1444C207843B2002BAE
:1032E00001DB01F056FD3300303318780222030071
:1032F000934300D1A8E23D4D3E4C2B7862322270C0
:1033000063702F79EA783F0217436A7912041743F2
:10331000AA7912063A436260222B01D101F079FBAF
:1033200000D951E1132B01D101F087F900D9E9E06F
:10333000092B01D100F08BFE2B4F00D9A7E0032B06
:1033400000D16DE368D8012B00D13FE2022B00D100
:1033500021E30223237077E2022B00D014E701223D
:103360000023244C224D22706370636068782B78B0
:10337000C3189B18DFB2FEF741FF2878FEF73EFF27
:103380002078FEF73BFF6078FEF738FFE079FEF724
:1033900035FFA079FEF732FF6079FEF72FFF207925
:1033A000FEF72CFF3800E1E6137090E7022323704C
:1033B0008DE7320039321378013B012B87D8736BCC
:1033C00014498B420DD85A1C18000849726301F049
:1033D000D4FD3300072230331A700D4B063A1A70B1
:1033E00075E7107073E7C0462CFFFF1FFC0200203A
:1033F0000CFEFF1F3C03002035040020FA030020D0
:10340000AA03002040F00F40F4030020F90300203D
:10341000340300206B030000052B01D100F0E9FB11
:1034200000D212E3062B94D1A878002801D000F036
:1034300007FE60606B78A22B01D100F08BFD01D9F3
:1034400000F049FC112B01D100F02EFD01D900F054
:1034500000FC082B01D100F006FD01D900F0DAFBD9
:10346000032B01D100F0E6FC00D9C5E3012B01D10B
:1034700000F0DEFC2D21012B01D800F0BBFC272140
:103480003D69002002F0DEFBA84700F0B6FC0C2BE3
:1034900001D101F0BCF81AD80A2B01D100F0DBFDF4
:1034A0000B2B00D055E7AB78022B01D001F0ABF825
:1034B0006878132801D900F0BDFEB54BA03080001C
:1034C000C118B44B0422C91801F007FDBCE10E2B52
:1034D00001D100F09EFE01D201F074F80F2B00D054
:1034E00037E7AB78012B01D100F0C9FE002B01D1E9
:1034F00000F0AFFE022B01D100F0C5FE04232370C3
:1035000000F0ABFE1A2B01D101F0C2FB30D8162B14
:1035100001D101F05AF9A0491AD8142B01D101F0B8
:10352000C8F8152B00D014E768780C2800D98BE177
:103530009A4B03F077F9E108E908F108F908010965
:10354000090912091A0922092A0932093A09420904
:10355000182B01D101F04AF901D801F039F96B7843
:103560002E2B01D901F08BFB01218D4AD1546BE147
:103570001E2B01D100F035FF0BD8874F1B2B01D13B
:1035800001F052F91C2B00D0E3E6002339373B70E1
:103590005AE1202B01D100F0CDFF01D800F088FFC7
:1035A0006878804C0A2801D901F0FAF97E4B03F0C3
:1035B00039F9F309010A050A090A0F0A150A190A55
:1035C0001D0A210A250A270A802B01D101F070FA71
:1035D00046D8412B01D100F05FFE25D8252B01D123
:1035E00001F068FB13D8232B01D101F01FFA242B23
:1035F00000D0AEE66878052800D925E1674B03F0D6
:1036000011F9220A280A2E0A340A3A0A400A272BFC
:1036100001D101F03CFA01D201F056FB402B00D061
:1036200097E601F0DFFE0FE1442B01D100F03CFEF4
:1036300009D8422B01D100F033FE432B00D088E69D
:1036400001F0D3FE00E1462B01D100F035FE01D29E
:1036500000F02EFE472B00D07BE601F0CAFEF3E01F
:10366000872B01D101F088FA4CD8832B01D101F0CE
:103670003EFA49490AD8812B01D101F01FFA822B69
:1036800000D066E6022339310B70DDE0852B01D1D5
:1036900001F062FA454801D801F04BFA0B00012510
:1036A0000C003B331D7043783C342370404B9A42EE
:1036B00001D901F056FA437B2B40029302982B006C
:1036C000002801D001F04EFA06AF3900100001F0D9
:1036D00054FC3B7863707B78A370BB78E370BB7954
:1036E00023717B7963713B79A371FB78E3716B463E
:1036F0001B7A23722A5D237A01359B182372082DC9
:10370000F8D1A1E08D2B01D101F074FA22491FD824
:10371000892B01D100F04CFE01D200F0D1FD8A2BA3
:1037200000D016E66A78234B002A01D000F068FF2B
:103730001A70EB78204A21491370214A1070002238
:103740000A7020490A70204A11780B4313707BE0FD
:10375000F22B01D100F0F8FDFF2B01D100F0EAFDC2
:103760009A2B00D0F5E5AB78002B01D001F001FBDE
:103770006B78012B01D101F0E2FA002B01D101F0AD
:10378000C7FA022B01D101F0E7FA032323705BE0B3
:1037900080FDFFFF480300202CFFFF1F04030020D3
:1037A000FE03002030030020440300200CFEFF1F16
:1037B0006B0300009C030020AB030020AA03002041
:1037C000FA030020350400209D030020AF78002F6D
:1037D00000D0DDE0BE4C2378002B07D0BD4B262166
:1037E0001A68380002F0F8F9AB78E7540127AC7892
:1037F000B94BE8781F552B791B0203436879000405
:103800000343A87900061843C317C0185840A30003
:10381000F358984727210200200002F0DDF92A79A9
:10382000EB7812021A436B79A8781B041A43AB7920
:103830001B0613430022934200DCA1E00197009293
:103840001300202102F07CF9A44C230030331B78B4
:10385000072B6ED1FEF73EFC626AA14D801AC2179B
:103860002B6880185040984208D99E4B1A78012A3C
:1038700001D101321A70FEF72DFC6062FEF72AFCBE
:10388000A26A6B68801AC21780185040984208D903
:10389000944B5A78012A01D101325A70FEF71AFC72
:1038A000A062FEF717FCE26AAB68801AC2178018A4
:1038B0005040984208D98B4B9A78012A01D10132A5
:1038C0009A70FEF707FCE06223007C331B78002B24
:1038D0002FD023007D331A78002A2AD11500814B7E
:1038E0008148995C022901D001F048FA91000958F9
:1038F0004F1C01D101F041FA7C487D4B00685833E0
:1039000018607C4800685860706B716398607A48F2
:103910000068D8603000383005781D61B56F5D6192
:10392000756F9D611A7700230370330001227D3388
:103930001A70230030331B78072B06D1220039324E
:103940001178022901D1033111706948016C0029F5
:1039500014D0072B12D1230039331B78012B0DD142
:103960000023656B994209D99A008218526CAA42C9
:1039700001D001F00AFA05233934237009B0F0BDF3
:103980000223009201932021130002F0D9F85BE793
:103990000423237058E7AF78002FF9D14C4C2378DB
:1039A000002B07D04B4B26211A68380002F014F97F
:1039B000AB78E7540127AC78474BE8781F552B7953
:1039C0001B020343687900040343A87900061843E7
:1039D000C317C0185840A300F35898472721020086
:1039E000200002F0F9F82A79EB7812021A436B7979
:1039F000A8781B041A43AB791B0613430022934299
:103A000007DD0223009201932021130002F098F8B1
:103A10001AE7019700921300202102F091F813E7B2
:103A2000AF78002FB4D101222B4B38001A70272118
:103A30003A0002F0D1F80223A8783A0001930097E7
:103A40003B00202102F07CF8FEE6AB780293002BCD
:103A50009ED16B780393012B50D0002B05D0022B05
:103A600000D190E003232370EEE61B4C2378002B5B
:103A700008D07A682721039802F0AEF86A46AB783E
:103A8000127BE254A878124C235C002B08D0114B17
:103A90008200D258262102F09FF80022AB78E2542F
:103AA0002B79EA781B0213436A79A878120413432E
:103AB000AA792D2112061A4302F08EF80022A87866
:103AC000130001920092202102F03AF8BCE6C046B1
:103AD0003404002030040020A90300202CFFFF1F25
:103AE000D8030020FE030020ACFFFF1F300300209E
:103AF0002C0000204403002004030020387B002811
:103B000039D001283CD0A878B14B1B5C002B09D0E0
:103B10008300FF187A68272102F05EF80022AB7854
:103B2000AB49CA54A878AB4F3B5C002B08D0AA4BDA
:103B30008200D258262102F04FF80022AB78FA54C6
:103B40002B79EA781B0213436A79A878120413438D
:103B5000AA792D2112061A43029BD7183A0002F0C7
:103B60003BF80022A878130001920092202101F076
:103B7000E7FF676068E62D2102F064F80290C2E773
:103B800021210298F8E7924C2378002B08D07A681C
:103B90002721029802F020F86A46AB78127AE254A4
:103BA000A8788C4C235C002B08D08B4B8200D25819
:103BB000262102F011F80022AB78E2542A79EB7842
:103BC00012021A436B79A8781B041A43AB792D2192
:103BD0001B0613431B18814A9B009A5801F0FCFFF7
:103BE0000022A878130001920092202101F0A8FF82
:103BF0002AE6FEF729FC27E6052B00D122E100D2B8
:103C00001CE1062B00D121E1072B00D126E1032383
:103C10002370F3E00C2B00D138E10CD80A2B00D133
:103C20002BE100D825E13521002002F00BF801231B
:103C300083436360E2E00E2B00D12BE100D227E149
:103C40000F2B00D12CE1102BE1D13D692521FFF78D
:103C500018FC1A2B00D143E11CD8152B00D12FE101
:103C600008D8132B00D127E100D821E13D692B2191
:103C7000FFF707FC172B00D128E100D222E1182B17
:103C800000D127E1192BC2D13421002001F0DAFF45
:103C90004007ECE01F2B00D12FE10CD81C2B00D1EA
:103CA00027E100D221E11D2BB1D100203D6901F0B7
:103CB000FBF9FFF7E9FB212B00D12CE100D223E136
:103CC0007F2B00D12DE18C2BA1D1002002F068F9CF
:103CD0000823181A91E0B92B00D193E144D8AB2BFB
:103CE00000D15FE121D8A62B00D142E10ED8A42B50
:103CF00000D136E100D830E1002002F06DF9002853
:103D000000D032E1A87802F08FF976E0A82B00D13C
:103D100040E100D23AE1A92B00D13FE1AA2B00D02B
:103D200075E7002002F020FA67E0B32B00D144E1F0
:103D30000BD8AD2B00D13CE100D236E1AE2B00D048
:103D400065E7002002F01EFA57E0B52B00D13FE1F5
:103D500000D236E1B62B00D13EE1B82B00D056E7B9
:103D6000002002F040F948E0C22B00D1DBE01CD873
:103D7000BD2B00D150E10AD8BB2B00D148E1132163
:103D8000BB2B00D829E1002002F0B0FA35E0BF2BB0
:103D900000D14DE100D241E1C02B00D14CE1C12B5B
:103DA00000D034E70E4B1B7A43E7CE2B00D1C6E0A0
:103DB00018D8C42B00D1BDE000D2B7E0C52B00D18C
:103DC000BBE0CC2B00D022E7002002F06CFA14E01C
:103DD000A903002034040020300400200803002040
:103DE000B4030020D62B00D1AEE018D83921D12B56
:103DF00000D00CE7002001F025FF6060C04B1B786D
:103E0000002B00D120E5BF4B616808221960BE4B32
:103E1000002900D016E119680A431A6014E5D72B6F
:103E200000D18EE0FF2B00D0F1E6B84B1B7E00E7FF
:103E30002121DFE73D692221FFF723FB3B697868F9
:103E40009847DAE77B69B24A1068F9E71021002049
:103E500001F0F8FE000AC0B2C000CEE71021002039
:103E600001F0F0FEF7E7352101F0ECFE8005C00F10
:103E7000C3E7002002F03EFBBFE73521002001F040
:103E8000E1FE0223034058425841B6E73421F5E7EA
:103E90003421C9E63421002001F0D4FEC006E6E753
:103EA0007D692421FFF7EDFA7D692821FFF7EAFA01
:103EB0007D692A21FFF7E5FA3D692321FFF7E1FA41
:103EC0002C2197E73D691521FFF7DBFA3D69332186
:103ED000FFF7D7FA3421002001F0B4FE0007C6E74F
:103EE000342101F0AFFE0005C1E7002002F066F8C2
:103EF00083E7002002F069F87FE71021002001F03D
:103F0000A1FE0003000F78E76E21002001F09AFE69
:103F10008005800D71E76E21002001F093FE000CFA
:103F20006BE73B7B85E63B69784A8DE7774A3B69DF
:103F3000506885E7774B1B687BE6774BFBE76F2183
:103F4000E3E7FEF76EFA58E71121002001F07AFE50
:103F5000400052E702F016F84FE7002002F03CF86C
:103F60004BE7002002F046F847E7A87802F049F84E
:103F700043E7002002F030F8002803D1A87801F0D0
:103F8000FAFF3AE7A87802F048F836E7002001F097
:103F9000EBFF32E7002002F003F92EE7002002F0E9
:103FA000DCF82AE702F0D2F827E7002002F0E3F875
:103FB00023E7002002F0FBF81FE7002002F038F8AA
:103FC0001BE76F21002001F03DFEC002C00E14E788
:103FD0004E4A3B69106933E71421002001F032FE9C
:103FE000011E12D04D4802F027FC6060AA78474BB2
:103FF00052019B181B7E002B00D0FFE6606802F088
:1040000085FAFAE601F0C5FFF7E6454B6360EDE798
:10401000002002F064F9F0E67121EBE600210800CF
:1040200001F010FE0423184000D1E6E6033B00E651
:10403000002002F04DF9E0E6002002F042F9DCE653
:104040000423E5E5196891431960FFF7FDFBFEF7CE
:1040500027FEFFF7F9FBAB78022B00D18AE0032B98
:1040600000D18CE0002B00D0CCE06B78542B5FD0DB
:1040700014D84B2B34D009D8422B2BD0442B2CD026
:10408000412B08D1274B9B78636055E04D2B30D0F6
:1040900029D3512B30D0032323704DE0812B5DD0E9
:1040A00008D8572B22D0802B45D0552BF3D11D4B50
:1040B000DB7BE9E7832B58D055D3842B57D0852B56
:1040C000E9D13A6A184B5343184A9B183B625B008C
:1040D0005B08D9E7134B1B78D6E7124B9B68D3E7F5
:1040E000104BDB78D0E70F4B5B78CDE70D4B1B799E
:1040F000CAE70C4B1B7BC7E70A4B5B7BC4E7C04698
:10410000340300203003002004030020B403002007
:104110003004002098030020D40300200024F40081
:10412000FFFFFF000CFEFF1F6D4EC641393000003F
:10413000CB4B9B7BA8E76160CA4B1B78002B01D15E
:10414000FFF782FBC84B616808221960C74B002942
:104150005AD119680A431A60FFF776FB04394A42BC
:104160004A416260E8E77B6B8EE7FB698CE7C04BF6
:104170001B6889E76B78BF4A9B009B5884E76B7884
:10418000272B2FD012D8022B24D007D8002B1FD0DA
:10419000012B00D07FE7B84B5B6875E71B2B1BD06A
:1041A0001C2B1CD0092B00D075E7C5E72B2B20D08A
:1041B00005D8B14A292B1AD017D9537D64E72D2B86
:1041C0001DD019D32E2B00D065E7AB4B5B7E5BE790
:1041D000A94BCDE7A84B81E7A74B1B7C54E7A64B27
:1041E0005B7C51E7A44B9B7C4EE7D37C4CE7137D73
:1041F0004AE7A14B9B7D47E79F4BDB7D44E79E4B06
:104200001B7E41E7042347E7196891431960FFF7D4
:104210001BFBAB78002B05D0022B0FD0042323709F
:10422000FFF712FB6B78002B04D11000FEF7AAF801
:10423000FFF70AFB03232370FFF706FB6878002AC9
:1042400003D1FEF793F8FFF7FFFAFEF790F8FFF7B8
:10425000FBFA6878FEF78CF86060824B1B78002BC5
:1042600001D1FFF7F1FA804B6168082219607F4B9A
:1042700000290CD119680A431A60FFF7E5FA68783B
:10428000FEF782F8E8E76878FEF77AF8E4E719685D
:1042900091431960FFF7D8FA01F0A5F8FFF7D4FAB7
:1042A00001F0A2F8FFF7D0FA01F0A0F8FFF7CCFA7E
:1042B00001F09DF8FFF7C8FA01F09AF8FFF7C4FA89
:1042C0006B78012B19D0002B05D0022B1ED00323B5
:1042D0002370FFF7B9FA0A0001203B321070604AE0
:1042E0003C3152780A70654A10685A1CC35C5354BA
:1042F0001300082AF9D1FFF7A7FA042263710C23EF
:10430000E271B632A2712371FFF79EFA0B0001220F
:104310003B331A70C022524B3C315B7852010B7018
:10432000574B58481C78181801330C549342F8D155
:10433000FFF78AFA544B9A4201D0FFF785FA01231E
:1043400045310B70FFF780FA6B78812B01D0FFF7B6
:104350007BFAAB78922B01D0FFF776FAAB79A32BDF
:1043600001D0FFF771FA6B79B42B01D0FFF76CFA2B
:104370002B79C52B01D0FFF767FAEB78D62B01D04C
:10438000FFF762FA2022414B5A6072B60022404B7E
:1043900040491A600123404A5B42D367C022520061
:1043A0008B503E4A3E4B1A60FDF76AFFFFF74CFA0E
:1043B0006B78002B01D0FFF747FAAB78002B01D0C8
:1043C000FFF742FA30498A4201D0FFF73DFA042252
:1043D00006A93448069300F080FDFDF751FFFFF772
:1043E00033FA6878092800D924E7AB78002B16D176
:1043F0002D4B8100CA501A4A927B002A01D1FFF747
:1044000023FA002801D1FFF71FFA284AD73080008D
:104410008118C918042200F060FDFFF715FAFF2B80
:1044200001D0FFF7B5FA204C00280FD1D825E1279D
:10443000AD00BF001D4B2800E918611804220435A7
:1044400000F04BFDBD42F5D1FFF7FEF9174BD73019
:104450008000C1186118042200F03FFDFFF7F4F955
:104460000CFEFF1F34030020300300200403002053
:104470003803002048030020D803002008FEFF1F57
:10448000F817000009E8FFFFD204000040F00F40D9
:1044900010E000E000E100E004E100E078563412B2
:1044A00000FEFF1FFE07000008030020A4FCFFFF22
:1044B0006878092800D9BDE6AB78002B19D1D24B1A
:1044C0008000C158D14B61601B78002B01D1FFF7F0
:1044D000BBF9CF4B08221960CE4B002904D11968D3
:1044E0000A431A60FFF7B0F9196891431960FFF7A2
:1044F000ABF9FF2B01D0FFF74BFAC34C00280FD1CB
:10450000D825E127AD00BF00C34B2800E91861188A
:104510000422043500F017FDBD42F5D1FFF794F9F0
:10452000BD4BD7308000C1186118042200F00BFD8C
:10453000FFF78AF96F78092F00D97BE6A87843B294
:10454000002B1EDAC30706D52121002001F07AFBDB
:10455000AD4ABF00B850B14B9B7B002B01D1FFF798
:1045600073F96878002801D1FFF76EF9AA4BD730AC
:104570008000C118A44B0422C91800F0AEFCFFF75C
:1045800063F9002801D0FFF703FA212101F05AFB5B
:104590009D4CBF00A14B38519B7B002B01D1FFF7F5
:1045A00053F96878002801D1FFF74EF9AA7811185D
:1045B000D7308018890009198000042200F08DFC92
:1045C000FFF742F9A878002801D0FFF7E1F96B78EE
:1045D000012B0CD0002B05D0022B0CD00323237011
:1045E000FFF732F9180001F091FAFFF72DF901F009
:1045F00097FAFFF729F901F09DFA6060FFF724F9B7
:104600000122FFF795F804232370FFF71DF9AB781B
:10461000022B0ED16878132800D90BE6804BA0300E
:104620008000C1187F4B0422C91800F08CFCFFF7F2
:104630000BF904232370FFF707F96878744C0928F5
:1046400015D802F0E5F805090C0F1E24272A2D07BE
:1046500023689A1822600AE023689A1AFAE7236806
:104660005A43F7E72068110002F070F920602168D2
:104670000822684B002917D119680A431A60FFF70E
:10468000E3F82068110002F047FA2160EFE72368A1
:104690001A40DFE723681A43DCE723685A40D9E76A
:1046A0002368DB432360E2E7196891431960FFF751
:1046B000CBF8574B5749186882420DDA03230A6832
:1046C0009A43013313430B600A68082300280FD173
:1046D00013430B60FFF7B8F8824204D106230A683F
:1046E0009A43053BEEE705230A689A43033BE9E753
:1046F0009A430A60FFF7A8F81B681B0701D4FFF76D
:10470000A3F84A63FFF7A0F81B681B0701D5FFF762
:104710009BF84A63FFF798F81B68DB0701D4FFF7A3
:1047200093F84A63FFF790F81B68DB0701D5FFF7A2
:104730008BF84A63FFF788F81B685B0701D4FFF723
:1047400083F84A63FFF780F818680523184201D1FF
:10475000FFF77AF84A63FFF777F81B689B0701D4E5
:10476000FFF772F84A63FFF76FF81B689B0701D1E8
:10477000FFF76AF84A63FFF767F81B68DB0601D4A6
:10478000FFF762F84A63FFF75FF81B689B0601D4E6
:10479000FFF75AF84A63FFF757F81B685B0601D426
:1047A000FFF752F84A63FFF74FF81B681B0601D466
:1047B000FFF74AF84A63FFF747F81B68DB0501D4A7
:1047C000FFF742F84A63FFF73FF87263FFF73CF8E0
:1047D0000B6D072B01D9FFF737F8581C08659B00B4
:1047E000486BCB1858654A63FFF72EF80B6D002B0A
:1047F00001D1FFF729F8013B0B659B00CB185B6DDE
:104800004B63FFF721F8C046080300203403002063
:104810003003002004030020A4FCFFFF0CFEFF1F58
:1048200080FDFFFF480300203B0038331B78002B3E
:104830000DD10A33511C13D1DF4A126853437B67F1
:10484000FDF748FC3B0001223833B8671A706878DE
:10485000032801D9FEF7F8FF01F0DAFF05194672C7
:104860005A437A67ECE7FDF735FCBB6FC01AC317F4
:10487000C01858407B6F984204D9002338373B70EA
:10488000FEF7E2FF7B6B013B7B63FEF7DDFFA87861
:104890003521802401F0D6F9A400044009D000237A
:1048A000C64A383711683B70103399431160FEF7E0
:1048B000CBFF7B6F002B12D0FDF70CFCBB6FC31A34
:1048C000DA179B1853407A6F934208D91023BB4ADA
:1048D000383711683C700B431360FEF7B5FF7B6BF4
:1048E000013B7B63FEF7B0FFA878352101F0AAF900
:1048F0000124044009D00023B04A383711683B70C6
:10490000103399431160FEF79FFF7B6F002B12D08D
:10491000FDF7E0FBBB6FC31ADA179B1853407A6FA1
:10492000934208D91023A54A383711683C700B43CD
:104930001360FEF789FF7B6B013B7B63FEF784FF0F
:10494000A878352101F07EF90224044009D0002323
:104950009A4A383711683B70103399431160FEF75B
:1049600073FF7B6F002B12D0FDF7B4FBBB6FC31A34
:10497000DA179B1853407A6F934208D910238F4A55
:10498000383711683C700B431360FEF75DFF7B6B9B
:10499000013B7B63FEF758FF1B682268D318236036
:1049A00021680822854B00292ED119680A431A6014
:1049B000FEF74AFF1B682268D31AF0E71B682268DB
:1049C0005343ECE72068196801F0C0FF2060E7E777
:1049D0002068196802F0A0F82160E1E71B682268EE
:1049E0001340DCE71B6822681343D8E71B68226882
:1049F0005340D4E71A68D2431A60D1E72268FBE734
:104A0000196822682160F7E7196891431960FEF779
:104A10001BFF694B1978E970597829719978DB780F
:104A20006971AB71FDF710FDFEF70EFF624B19784F
:104A3000E970597829719978DB786971AB71FEF763
:104A40002FF9FEF701FF0F2219680A401A60FEF7DE
:104A5000FBFE1022196891431960FEF7F5FE202233
:104A6000196891431960FEF7EFFE402219689143DF
:104A70001960FEF7E9FE8022196891431960FEF77C
:104A8000E3FE19684E4A0A401A60FEF7DDFEAB7875
:104A9000002B01D0FEF77CFF6B78092B01D9FFF7C3
:104AA000C9FB454A9B001168464A9950FEF7CCFE67
:104AB0003300002239331A70FEF7C6FE6B78002BE4
:104AC00005D0012B08D003232370FEF7BDFE012380
:104AD00039310B70FEF7B8FE3B48824201D9FEF730
:104AE00057FF0800393003704A63FEF7ADFE32000D
:104AF00000237C321370320001257D3213701A00BE
:104B0000324833496D429C00CA54013325502F2B43
:104B1000F9D1304B19001A655A6338331A70264B95
:104B200039311A602C4B0A701A60244B1A60FEF758
:104B30008BFE437B9B070BD4234B9A4201D9FEF794
:104B400027FF042339310B70244BDA63FEF77CFE18
:104B500008232370FEF778FE002339310B70FEF72F
:104B600073FE2B0000223C315A540133082BFBD139
:104B70000B780B72FEF768FE6878032801D9FEF700
:104B800063FE144B01F044FE020D2C3138331B78C8
:104B9000E171A371114BDB6B1A0A62712371FEF78D
:104BA00053FE1A00383212785B6BA2711A0AE17157
:104BB00062712371FEF748FE3003002004030020D9
:104BC000FFFEFFFF080300206B030000ACFFFF1F88
:104BD000FE0300202CFFFF1F440300202C000020B8
:104BE000844B1B686360FEF72FFE834B1B6863607A
:104BF000FEF72AFE687803283DD801F009FE170267
:104C00002E387E4C00212500236C4435994201D179
:104C1000FEF71AFE8800475997421CD12200013B3B
:104C20004432994211D32364FEF70EFE734B196C84
:104C3000042906D8481C890018645B185A64FEF7DA
:104C400003FE09232370FEF7FFFD15186D6801317F
:104C500085500430E5E70131D8E70022674B1A643C
:104C60005A649A64DA641A655A65FEF7EDFD052305
:104C70006360FEF7E9FD03232370FEF7E5FDFF2BDC
:104C800001D0FFF7D7FA7C31FE3B0B70FEF7DCFD5D
:104C90006B782E2B04D80021594AD154FEF7D4FD4D
:104CA000FF2B01D0FFF7C6FA330000227C331A70C5
:104CB000FEF7CAFD6B782E2B01D9FFF7BBFA5149DD
:104CC0009B005A50FEF7C0FD4C4B4A4A996D11604B
:104CD000D96D494A11601A6E596E72634A4A116061
:104CE000682132005918097838321170DA6E583359
:104CF000B2679A6972671B7F414AD15C002901D073
:104D00000121D1540022414B7D331A70FEF79CFDE6
:104D10003F4B9A420FD101F03EFC01F09BFC041C7A
:104D2000D8203C4B40019847D820210040013A4B05
:104D30009847FEF789FD04232370FEF785FD01F0F7
:104D400089FC02F05DFD0022344B02F0A5FA02F06E
:104D500023FD6060FEF778FD01F082FC02F050FD5B
:104D600000222E4B02F098FA02F016FD6060FEF76A
:104D70006BFD04232370FEF767FD9D5401322F2A3B
:104D800001D0FEF7AEFDFEF7D4FD0133DBB2FEF736
:104D9000E9FD0221303633788B4301D1FEF7EEFD79
:104DA0001F4DE37868702179144E09021943637925
:104DB000F06B1B041943A3791B060B436B60194B63
:104DC000984210D8210000F0CFF82100F06B00F0DD
:104DD000F8F80723002803D0F36B0133F36365234E
:104DE0002B70FEF7CBFD07232B7000231370FEF70B
:104DF000C5FDC04630030020440300202C000020E5
:104E0000FE030020ACFFFF1F040300202CFFFF1F48
:104E10004E61BC0035FEFF1F6DFEFF1F0088C340C2
:104E20003C0300206B03000080230A490A4ADB038D
:104E3000885803438B505C22084BDA7000229A702A
:104E400022325A70C023064A9B009361D361054AFF
:104E50001360704700700440341000000060074089
:104E60000090044000A0044070B5002813D10B4C02
:104E70000B4B25002030986026780642FCD0A171AB
:104E8000297849B20029FBDAA879C0B2002A01D0FA
:104E900020225A6070BD0020FCE7C0460060074039
:104EA00000F00F4010B5FDF715F90400FDF712F9F9
:104EB000001BC317C01858400628F7DD10BD07B502
:104EC000020A01AB1A705870997003221900A020D1
:104ED00000F02CFBFFF7E6FF07BDF0B51500002240
:104EE00014008DB00191AC4201D10DB0F0BD1F276F
:104EF000019E03A9365D8B189E70531CC6183E4256
:104F000002D06F1EBC420AD1030A48700332A020AF
:104F10000B7000F00BFBFFF7C5FF300000230134DE
:104F20001A00E0E713B501AC030A60702100022209
:104F3000A020237000F0FAFA02222100A02000F045
:104F40001BFB207816BD37B515000C0001A9030A1C
:104F500048700222A0200B7000F0E8FA2A0021001D
:104F6000A02000F009FB37BD0722802310B5504375
:104F70001B01C018FFF7B1FF10BD0722802310B539
:104F800050431B01C018FFF7DEFF10BD00231A00BD
:104F900070B58AB001AD5A550133222BFBD1802662
:104FA0000024B601230A6C7022222900A02020349C
:104FB0002B7000F0BBFAFFF775FFB442F2D10AB0D4
:104FC00070BD0722802313B550431B01C0180C008D
:104FD0006946FFF7B8FF6B461A78237800209A429B
:104FE0001BD16B465A7863789A4216D16B469A78F1
:104FF000A3789A4211D16B460198DB78000222799E
:105000000343E07812020243607900040243A0796E
:1050100000061043181A4342584116BD704773B535
:105020006B469C1D022221001848FFF78CFF228846
:10503000174B184D9A4203D1174B1B78002B19D0F0
:1050400000260222210011482680FFF746FFFFF7C5
:105050009DFF202229003000FFF73FFF20220F494B
:105060004020FFF73AFF0E4B022221000748238021
:10507000FFF733FF290020220020FFF764FF2022E2
:1050800008494020FFF75FFF73BDC046FE070000E0
:10509000A5A500000CFEFF1FB0030020C079000092
:1050A000A5A5FFFFB4030020014B8000C058704746
:1050B000A4000020F7B5B14EB368002B13D0B04D5B
:1050C0002C78002C0FD1FDF705F8AE4B1B68C01AE9
:1050D000C317C0185840B368984204D90123200070
:1050E0002B7001F0F3F9A84C207901F00AFA00289E
:1050F00001D001F017F9FCF7EDFF63689B00E3189E
:105100009B68C01AC317C01858400A2824DDFCF752
:10511000E1FF21210600207900F094FD636807007B
:105120009B00E5180093EB68C01A02F065F8AB68C5
:105130000190F01A02F060F8011C019801F02CFDBA
:1051400002F05EFB914B924A02F0A6F802F024FBBB
:10515000009BAE60E050EF608B4C3521207900F071
:1051600071FD40260700064006D0207901F0AEF917
:105170000122884B61685A546068874D4301EB18DF
:105180001B69002B4DD0C0B2222100F05BFD63688B
:10519000C217801850405A01AD182A69904240D970
:1051A000E218127C002A0FD1DDB23421280000F071
:1051B00049FD8022D20002433421280000F00CFD7A
:1051C00001226368E3181A74657C002D0AD1E8B2E5
:1051D000FDF7CEF823001233E8540135082DF6D13F
:1051E000012363740025E8B2FDF7C2F823001233EF
:1051F000EA5C824232D0E854684B5B199B7CDBB29C
:10520000022B22D0032B03D0012B27D1002825D03D
:105210002B00634A2733D15C01291FD10131D154BE
:105220001CE0656863191B7C002BCDD0EDB23421E6
:10523000280000F007FD5B4A34210240280000F0FE
:10524000CBFC63680022E318BDE7002806D12A00E2
:1052500053492732885C012800D18B540135082D31
:10526000C1D10120390063680140E218002911D042
:10527000917E00291ED19076484AD218127C0242B3
:1052800018D08340464A1B33D15C814212D102219F
:10529000D1540FE0907E00280CD0917602213F4A35
:1052A000D218127C0A4205D05B003D4A1B33D05C09
:1052B0000128EDD00222380063681040E118002870
:1052C0004AD0C87E00280DD10130C8763349C918AC
:1052D000497C014206D00E3383403149C85C012825
:1052E00000D1CA5480231F4044D063682C4A033342
:1052F000D15C012901D10131D154002E09D063685C
:10530000274A0F33D15C012901D10131D154002F3B
:1053100014D025486168037801221D000D41154213
:105320000CD015008D402900204D2970204D2A7089
:10533000204A1278002A01D18B4303702079C022C1
:10534000352100F049FC207900F098F963680133B9
:10535000002B0DDC6360F7BDCD7E002DC2D0C8767A
:105360000E49C918497C1142BCD00E335B00B4E72A
:105370000023EFE7002EE1D0C1E7C0460CFEFF1F7F
:10538000F9030020F4030020A40000204D629040A7
:10539000FCA9F1D2B1030020B4030020D8030020FF
:1053A000FE030020FFFBFFFFAB030020AA03002049
:1053B000350400209C030020704710B5FCF78AFEDE
:1053C000064C2368C01AFA235B00984205D90222D2
:1053D000034BDA60FCF77EFE206010BD380400202D
:1053E00040F00F40704770477047704770477047F4
:1053F0007047704710B502243A4AD378100023430F
:10540000D370394B1978C9B2A14243D0032937D0A0
:10541000012910D15C789878844218D2D07808425B
:105420000AD159785C68C9B2481CC0B2587061187A
:105430000B78DBB2137110BD20249078A0439070DC
:105440009078103CA04390701972002216E0597AAF
:105450009078C9B2002908D12024A0439070907898
:10546000103CA04390701970E5E70421014391704E
:10547000997AC9B2117100225A7203321A70DAE7AE
:1054800010209178814391701279D968D2B20A7054
:105490001C70D0E71C7C597C8C421ED25A7C197C33
:1054A000521A012A05D1202182788A438270002273
:1054B0001A705A7C197C521A022A03DC082281785D
:1054C0000A4382701A7CDC68D2B2511CC9B21974CA
:1054D0000379A218DBB21370ADE7202091788143E5
:1054E0009170B2E700600640C000002040230B49E5
:1054F0000B4A10B5885803438B508022094B920009
:10550000DA601A61084BED3AFF3A5A70AC329A7081
:10551000002208205A7101F0B9F810BD0070044053
:105520003410000000A004400060064030B50024A4
:1055300008250F4BD2B21C725C729A705C700D4AD7
:10554000013459601C709178A043A94391701021D7
:105550009578294391702021957829439170107195
:105560001A78002AFCD1187A43425841C0B230BDA3
:10557000C00000200060064010B50024104BD2B2DD
:105580001C725C725A7403221C741A700D4AD96022
:1055900091780834A143917010219478214391703F
:1055A00020219478214391700121084310711A78C9
:1055B000002AFCD1187A43425841C0B210BDC046FF
:1055C000C00000200060064070B5144C0125E36067
:1055D0006B4600261B7CD2B226726572A270667082
:1055E00063742B006160082103432674A3720C4B83
:1055F00025709A78A8438A439A70102299780A43B2
:105600009A70202299780A439A7018712378002B97
:10561000FCD1207A43425841C0B270BDC000002086
:105620000060064073B5124E0400335C0D00002B81
:1056300007D0104B8200D258262100F0CDFA00236B
:105640003355EB17EA185A402721200000F0C4FA1E
:105650000123094A13550022954207DD0193009268
:1056600013002021200000F06BFA73BD0223F5E740
:105670003404002030040020A9030020F0B53521B7
:1056800089B0040000F0DEFA0590CA4865014119AE
:10569000059A0B7A5608496801225F0625D51640FF
:1056A0003700059E16402A580796524206924A42F3
:1056B00004923F261E405BB22000002B1DDA00F052
:1056C00019FF030058425841C3B2701E03930728C4
:1056D00000D985E1B84D01F0A5F8150015001500B9
:1056E00015001101110111011101059F164017400C
:1056F0002A58079606920491DBE700F0FBFE431E52
:105700009841E1E7285D01380E2800D968E101F0F1
:1057100089F80F001E002D003B004B005300620073
:1057200070009D00C000C5006701F000EF01EA01B4
:105730003421200000F086FA0122A300EB18586003
:105740009E4B023E1A5596421BD802231AE0A30034
:10575000EB185B6802221A433421200000F03CFA67
:1057600006992000FFF75EFF03230BE0079B002B49
:1057700000D135E12121200000F064FA904BA20015
:10578000D05004232B552BE1A300EB185B680122BA
:105790001A433421200000F01FFA069B20005942D2
:1057A000FFF740FF0523EDE7002F00D118E12000AF
:1057B00000F08CFE0623E5E7A300EB185A680323EC
:1057C000342120009A4300F007FA04992000FFF7E3
:1057D00029FF0723D6E7002F00D001E13900200080
:1057E000FFF720FF049B20005942FFF71BFF08230F
:1057F000C8E7002F00D1F3E02121200000F022FAB9
:10580000060000212000FFF70DFF6D49A3005A5844
:105810002000921B5A50EB185A68032334219A43F4
:1058200000F0DAF9049A2721200000F0D5F93200BF
:105830002D21200000F0D0F9002220211300019238
:105840000092200000F07CF909239BE7059B9B0553
:1058500000D4C5E02121200000F0F4F9594B0021CB
:1058600018602000FFF7DEFE00222D21200000F04E
:10587000B3F900222121200000F0AEF9033E0022FE
:105880003921200000F0A8F9012E35D8049B594297
:10589000BBE0002F00D1A3E00B2373E7002F00D063
:1058A0009EE02121200000F0CDF939000600200003
:1058B000FFF7B8FEA300EB185A68032334219A437C
:1058C000200000F089F9049A2721200000F084F9D3
:1058D000F20F921952102D21200000F07DF93B00AB
:1058E000019700973A002021200000F029F90D23AC
:1058F00048E7059B9B0573D50E2343E7285D0138D8
:105900000E286DD800F08EFF0F00210033004300F9
:1059100060006C006E006C006C009A00A5008600B0
:10592000D000F400EF000122244B342120001A554E
:1059300000F088F9A300EB1858600223063E9E434E
:10594000F6B2002E00D01CE71CE7062E06D1A300FD
:10595000EB185A6803239A431300FBE6082E00D085
:10596000FEE6A300EB185A6803239A43F4E6731F7C
:10597000012B07D8079B002B04D0062E00D100E78F
:105980000F23FFE6039B002B2AD00C23FAE6052EFB
:1059900006D1A300EB185A6803239A431300F6E6D6
:1059A000072E00D0F9E6A300EB185A6803239A43A8
:1059B000EFE6C046B4030020D4000020A903002075
:1059C00098030020D4030020731F012B04D8002F5C
:1059D00002D0052ED4D1B8E6039B002B00D0F8E608
:1059E00009B0F0BD039B002BFAD1073E012E0BD965
:1059F000A300EB185A6803239A43130002223421B0
:105A00001A43200000F0E8F804992000FFF70AFE8E
:105A10000A23B7E6039B002BE2D1073E012E00D8F4
:105A200034E7A300EB185A6803239A4313000122BA
:105A300034211A43200000F0CFF827E7039B002B06
:105A4000CED02121200000F0FDF8A300EB189860D3
:105A500022E7039B002BC3D12121200000F0F2F8A4
:105A600003230500274FA600BE19726834219A430C
:105A7000200000F0B1F8049A2721200000F0ACF8D3
:105A8000B2682D21AD18EA0F52195210200000F013
:105A9000A3F8039B2021019300931A00200000F03B
:105AA0004FF80D233B559BE7059B9B0598D50E238F
:105AB000212120002B5500F0C5F8134B0021186060
:105AC0002000FFF7AFFD200000222D2100F084F818
:105AD00020000022212100F07FF80022392120003F
:105AE00000F07AF87CE700212000FFF79BFD03E738
:105AF000A300EB185A683421200000F06DF8002351
:105B000040E6C046D4000020D4030020034B1A5CBA
:105B1000002A01D101321A547047C046D400002037
:105B2000034B1A5C002A01D00F221A547047C0465A
:105B3000D4000020014B185C7047C046D400002000
:105B4000F7B51F0008AB1D7809AB1B780600009362
:105B50007F230B4014000193352B10D114022743EF
:105B60003F023D43009B2D022B431D00184A353652
:105B7000B600184FB3583D40AB43B350F7BD802338
:105B8000002219431000FFF76FF9002221001000D6
:105B9000FFF76AF9002239001000FFF765F90022CB
:105BA00029001000FFF760F924020122009900206B
:105BB000FFF75AF92743019B3F029E193D43009B83
:105BC0002D022B431D00024BB600F550D6E7C04610
:105BD000E0000020CC100000F8B57F24070015007D
:105BE0000C40164E352C08D10400154B3534A4005A
:105BF0001D403359AB433351F8BD80230022194374
:105C00001000FFF731F90022290E1000FFF72CF9E0
:105C100000222914C9B21000FFF726F90022291228
:105C2000C9B21000E419FFF71FF9A400E9B201227C
:105C30000020FFF719F93551DEE7C046E0000020EB
:105C4000CC10000070B57F242E4B0C401B5D05006E
:105C5000002B52D0002221001000FFF705F901238C
:105C6000184201D0284A5355002211001000FFF7B6
:105C7000FBF8002211001000FFF7F6F800221100D7
:105C80001000FFF7F1F8002101220800FFF7ECF8FF
:105C9000002211001000FFF7E7F8002211001000A9
:105CA000FFF7E2F80022060211001000FFF7DCF80F
:105CB0000022064311001000FFF7D6F8002136023B
:105CC000064301220800FFF7CFF836023043352C97
:105CD00009D12C000D4A3534A400A1580C4B0B40BF
:105CE0001843A05070BDDF23223C1C42FAD10302AE
:105CF000F8D5FF231B061843F4E72418034BA40030
:105D0000E058EFE7E0790000E0020020E00000202A
:105D1000CC10000070B50D006C210400FFF792FF5D
:105D200002000F20054082432A436C212000FFF728
:105D300053FF70BD70B50C006C210500FFF782FFAA
:105D40007023220198431A4002436C212800FFF778
:105D500043FF70BD70B50C006C210500FFF772FFAA
:105D6000E203C02464022240034C6C212040024321
:105D70002800FFF731FF70BDFF7FFEFF70B50C00FC
:105D80006C210500FFF75EFF2205F0242404224069
:105D9000034C6C21204002432800FFF71DFF70BD1B
:105DA000FFFF0FFF70B50C006C210500FFF74AFFE5
:105DB0002206F02424052240034C6C21204002439B
:105DC0002800FFF709FF70BDFFFFFFF070B50D0061
:105DD0006C210400FFF736FF002D07D08022D2058A
:105DE00002436C212000FFF7F7FE70BD014A02401C
:105DF000F7E7C046FFFFFFBF70B50D006C21040040
:105E0000FFF720FF002D07D08022120302436C21F0
:105E10002000FFF7E1FE70BD014A0240F7E7C046EF
:105E2000FFFFF7FF70B50D006C210400FFF70AFFBC
:105E3000002D07D08022D20202436C212000FFF700
:105E4000CBFE70BD014A0240F7E7C046FFFFFBFFF3
:105E500070B50D006C210400FFF7F4FE002D07D093
:105E60008022D20102436C212000FFF7B5FE70BDF5
:105E7000014A0240F7E7C046FFBFFFFF70B50D00C3
:105E80006C210400FFF7DEFE002D07D08022920176
:105E900002436C212000FFF79FFE70BD014A0240C3
:105EA000F7E7C046FFDFFFFF70B50D006C2104006F
:105EB000FFF7C8FE002D07D08022520102436C215B
:105EC0002000FFF789FE70BD014A0240F7E7C04697
:105ED000FFEFFFFF70B50C006C210500FFF7B2FE6D
:105EE00023070DD57023802298431201104322010D
:105EF0007024224002436C212800FFF76DFE70BD24
:105F0000014A1040F3E7C0468FF7FFFF70B50C0061
:105F10006C210500FFF796FEE201F024E400224028
:105F2000034C6C21204002432800FFF755FE70BD52
:105F30007FF8FFFF10B5FFF7E9FF10BD70B50D004A
:105F40006C210400FFF77EFE002D07D08022920214
:105F500002436C212000FFF73FFE70BD014A024062
:105F6000F7E7C046FFFFFDFF10B56C21FFF76AFEA3
:105F70000F23184010BD10B56C21FFF763FE4006DB
:105F8000400F10BD10B56C21FFF75CFEC003800F01
:105F900010BD10B56C21FFF755FE0002000F10BDBB
:105FA00010B56C21FFF74EFE0001000F10BD10B5BB
:105FB0006C21FFF747FE4000C00F10BD10B56C21EB
:105FC000FFF740FE0003C00F10BD10B56C21FFF7B6
:105FD00039FE4003C00F10BD10B56C21FFF732FE33
:105FE0004004C00F10BD10B56C21FFF72BFE8004DC
:105FF000C00F10BD10B56C21FFF724FEC004C00F08
:1060000010BD10B56C21FFF71DFE02004006400FC9
:10601000130501D50823184310BD10B56C21FFF7F7
:1060200011FE4005000F10BD10B5FFF7F6FF10BDC3
:1060300010B56C21FFF706FE8003C00F10BD70B5D0
:106040000C006D210500FFF7FDFD60236201984300
:106050001A4002436D212800FFF7BEFD70BD70B5E8
:106060000C006D210500FFF7EDFD6203C024E40183
:106070002240044C6D21204002432800FFF7ACFD74
:1060800070BDC046FF9FFFFF70B50C006D2105007D
:10609000FFF7D8FD2202F02424012240034C6D2199
:1060A000204002432800FFF797FD70BDFFF0FFFF7F
:1060B00070B50D006D210400FFF7C4FD02000F2034
:1060C000054082432A436D212000FFF785FD70BD06
:1060D00070B50D006D210400FFF7B4FD044A2D04D6
:1060E00002402A436D212000FFF776FD70BDC046B7
:1060F000FFFF00FF70B50D006D210400FFF7A2FD4A
:10610000002D07D08022120202436D212000FFF7EC
:1061100063FD70BD014A0240F7E7C046FF7FFFFF05
:1061200070B50D006D210400FFF78CFD002D07D028
:106130008022520402436D212000FFF74DFD70BD07
:10614000014A0240F7E7C046FFFFFFFE10B56D2190
:10615000FFF778FD4006800F10BD10B56D21FFF7E9
:1061600071FD4004800F10BD10B56D21FFF76AFD71
:106170000005000F10BD10B56D21FFF763FD0F2363
:10618000184010BD10B56D21FFF75CFD0314D8B2A7
:106190001B0601D5014B184310BDC04600FFFFFF91
:1061A00010B56D21FFF74EFD0004C00F10BD10B5F6
:1061B0006D21FFF747FDC001C00F10BD70B50C0089
:1061C00070210500FFF73EFD054A702110400322B3
:1061D0002240120502432800FFF7FEFC70BDC046B6
:1061E000FFFFCFFF70B50D0070210400FFF72AFDFF
:1061F000002D07D080221203024370212000FFF7F8
:10620000EBFC70BD014A0240F7E7C046FFFFF7FF15
:1062100070B50D0070210400FFF714FD002D07D0AC
:106220008022D202024370212000FFF7D5FC70BD0E
:10623000014A0240F7E7C046FFFFFBFF70B50C00C4
:1062400070210500FFF7FEFC054A70211040032273
:106250002240120402432800FFF7BEFC70BDC04676
:10626000FFFFFCFF70B50C0070210500FFF7EAFC92
:10627000044A24020240224328007021FFF7ACFCAC
:1062800070BDC046FF00FFFF70B50C007021050017
:10629000FFF7D8FCFF2302009A4328002243702115
:1062A000FFF79AFC70BD10B57021FFF7CBFC8002A0
:1062B000800F10BD10B57021FFF7C4FC0003C00FA4
:1062C00010BD10B57021FFF7BDFC4003C00F10BD1D
:1062D00010B57021FFF7B6FC8003800F10BD10B51C
:1062E0007021FFF7AFFC000AC0B210BD10B57021DD
:1062F000FFF7A8FCC0B210BD70B50E006F211500ED
:106300001C00FFF79FFC002E02D043039B0D33605F
:10631000002D02D0C302DB0E2B70002C01D0000E2A
:10632000207070BDD8235B0137B51868514C431CF1
:10633000012B00D899E0011C606000F01DFE862151
:10634000C90500F019FEA060FBF7C4FE0500FBF7CD
:10635000C1FE401BC317C01858400928F7DD0121B2
:106360000020FFF76FFC582300220193563B1000DA
:1063700000936C210133FFF7E3FB012500220F237B
:10638000100000931021083B0195FFF7D9FB3A4A12
:1063900070210020FFF720FC002220211000FFF7D1
:1063A0001BFC00222D211000FFF716FC00222121EA
:1063B0001000FFF711FC2A0023210020FFF70CFC3E
:1063C000A1682E4800F0E8FB00F0F6FE2421020050
:1063D0000020FFF701FC6168284800F0DDFB00F0B9
:1063E000EBFE252102000020FFF7F6FBA168244800
:1063F00000F0D2FB00F0E0FE262102000020FFF7B3
:10640000EBFB61681E4800F0C7FB00F0D5FE2721BA
:1064100002000020FFF7E0FBA168194800F0BCFB78
:1064200000F0CAFE282102000020FFF7D5FBA1687A
:10643000124800F0B1FB00F0BFFE2A21020000204C
:10644000FFF7CAFB61680F4800F0A6FB00F0B4FE3E
:106450002B2102000020FFF7BFFB29000020FFF7DF
:10646000F1FB284000D1207037BD074B6360074B1C
:10647000A36069E7E0020020800405000000C84630
:10648000000048470000204177BE3F3FC39D8F4238
:1064900070B5064C2418217B002905D1657BFFF7D8
:1064A00039FC01236573237370BDC046E0020020F0
:1064B00010B5054B1B181A7B002A04D00022597B0B
:1064C0001A73FFF727FC10BDE002002037B5012545
:1064D000074B002227211D540400FFF77DFB0022FB
:1064E00001950092130020212000FFF729FB37BD02
:1064F000A903002010B50421FFF7A4FB01231840D5
:1065000010BD014B185C7047E002002010B500F090
:1065100073FE034B596800F03FFB00F04DFE10BDC9
:10652000E002002010B500F067FE034B996800F010
:1065300033FB00F041FE10BDE002002070B50024E6
:106540000500A04214D000F057FE0B4B596800F034
:1065500013FD061C00F030FE040000F04DFE011C8F
:10656000301C00F0EBFA002802D1002D02DB0134D0
:10657000200070BD013CFBE7E002002010B500F0F8
:106580003BFE034B996800F0F7FC00F015FE10BDD0
:10659000E0020020704773B50020FFF7E5FC002102
:1065A00005000800FFF7B6FB264A26210020FFF76A
:1065B00013FB254A27210020FFF70EFB00200123B3
:1065C00000900193020003002021FFF7B9FAFBF7C6
:1065D00081FD0400FBF77EFD001BC317C018584067
:1065E0006328F7DDFBF776FD212106000020FFF789
:1065F00029FB0400FBF76EFD831BDA179B18534041
:10660000632BF7DD21210020FFF71CFB0022060091
:1066100027211000FFF7E0FA29000020FFF77AFB9E
:10662000301B00F0E9FD094900F0B6FA084C011CE6
:10663000606000F0A1FC8621C90500F09DFCA0600F
:1066400073BDC04660EA00001027000000007A44D5
:10665000E0020020014B58687047C046E00200206D
:10666000014B98687047C046E002002000BE7047AA
:1066700010B5044B044A9A6000F05AF800F096F8FE
:1066800010BDC04600ED00E0001C0000202801DD28
:10669000C0467047074B184004D5202301385B42A1
:1066A000184301300123C0218340034A490053505D
:1066B0001360EEE71F00008000E100E0202801DD0C
:1066C000C0467047064B184004D5202301385B4272
:1066D0001843013001238340024AD367F1E7C046E3
:1066E0001F00008004E100E010B503291BDC202816
:1066F00019DC0322C31713401B18FC329B108901BD
:106700001340094C1140094A9B001B19104004D545
:1067100004220138524210430130C0B2C00081400F
:106720001A681143196010BD00E400E00300008006
:10673000082310B5154A9178194202D091780B437D
:106740009370882100222220114B49015A5011498F
:106750000870802010494002585019680F480140C5
:106760001960C0210E4889041C582143195080210A
:106770000C4B1A7219767F391A7059700A490A70CF
:106780000C3299791142FCD110BDC04600D00740AF
:106790000070044000E0074044100000FFFFF3FFDA
:1067A0000410000000400640005006400C2210B5C6
:1067B000114B997911421CD099791140042911D1BA
:1067C0001B7A03391B075B0F99400C4800F034F823
:1067D0000B4B0C4AD158090F013100F02DF80A4B30
:1067E000186010BD9B791340082BFAD1802000025D
:1067F000EEE70648ECE7C0460040064000127A008B
:10680000441000000070044030FEFF1F006CDC02EA
:1068100002B4714649084900095C49008E4402BC33
:106820007047C04603B47146490840004900095A00
:1068300049008E4403BC7047002243088B4274D346
:1068400003098B425FD3030A8B4244D3030B8B4271
:1068500028D3030C8B420DD3FF22090212BA030C7A
:106860008B4202D31212090265D0030B8B4219D35B
:1068700000E0090AC30B8B4201D3CB03C01A52417B
:10688000830B8B4201D38B03C01A5241430B8B42C3
:1068900001D34B03C01A5241030B8B4201D30B03AC
:1068A000C01A5241C30A8B4201D3CB02C01A5241D3
:1068B000830A8B4201D38B02C01A5241430A8B4296
:1068C00001D34B02C01A5241030A8B4201D30B027F
:1068D000C01A5241CDD2C3098B4201D3CB01C01A99
:1068E000524183098B4201D38B01C01A52414309A3
:1068F0008B4201D34B01C01A524103098B4201D391
:106900000B01C01A5241C3088B4201D3CB00C01AFD
:10691000524183088B4201D38B00C01A5241430875
:106920008B4201D34B00C01A5241411A00D201469A
:10693000524110467047FFE701B5002000F0F0F823
:1069400002BDC0460029F7D076E7704703460B43E7
:106950007FD4002243088B4274D303098B425FD358
:10696000030A8B4244D3030B8B4228D3030C8B4284
:106970000DD3FF22090212BA030C8B4202D312126A
:10698000090265D0030B8B4219D300E0090AC30B3F
:106990008B4201D3CB03C01A5241830B8B4201D3EC
:1069A0008B03C01A5241430B8B4201D34B03C01AD5
:1069B0005241030B8B4201D30B03C01A5241C30A4D
:1069C0008B4201D3CB02C01A5241830A8B4201D3BE
:1069D0008B02C01A5241430A8B4201D34B02C01AA8
:1069E0005241030A8B4201D30B02C01A5241CDD24D
:1069F000C3098B4201D3CB01C01A524183098B4298
:106A000001D38B01C01A524143098B4201D34B0180
:106A1000C01A524103098B4201D30B01C01A5241E3
:106A2000C3088B4201D3CB00C01A524183088B426A
:106A300001D38B00C01A524143088B4201D34B0053
:106A4000C01A5241411A00D20146524110467047C5
:106A50005DE0CA0F00D04942031000D340425340CA
:106A600000229C4603098B422DD3030A8B4212D38A
:106A7000FC22890112BA030A8B420CD389019211BC
:106A80008B4208D3890192118B4204D389013AD0F9
:106A9000921100E08909C3098B4201D3CB01C01ACE
:106AA000524183098B4201D38B01C01A52414309E1
:106AB0008B4201D34B01C01A524103098B4201D3CF
:106AC0000B01C01A5241C3088B4201D3CB00C01A3C
:106AD000524183088B4201D38B00C01A5241D9D254
:106AE00043088B4201D34B00C01A5241411A00D2D5
:106AF0000146634652415B10104601D34042002BD1
:106B000000D54942704763465B1000D3404201B54F
:106B1000002000F005F802BD0029F8D016E7704704
:106B20007047C0468446081C6146FFE71FB500F069
:106B3000E1F9002801D40021C8421FBD10B500F0C2
:106B400073F94042013010BD10B500F0D3F90028B0
:106B500001DB002010BD012010BDC04610B500F0C3
:106B6000C9F9002801DD002010BD012010BDC0467C
:106B700010B500F07FF9002801DC002010BD0120D5
:106B800010BDC04610B500F075F9002801DA0020EC
:106B900010BD012010BDC046F0B557464E46DE463A
:106BA0004546E0B544024300C60F83B00F1C640A9B
:106BB0001B0EB24653D0FF2B27D08022E400D20414
:106BC00014437F22524290469844002399469B46A4
:106BD0007D027800FB0F6D0A000E009324D0FF2881
:106BE00046D080230021ED00DB041D437F3847465B
:106BF000381A4F460F43BF00B9463300009A874FFB
:106C000053404A46BA5801939746002C4ED1082368
:106C10009946F7339846FD3B9B467D027800FB0F73
:106C20006D0A000E0093DAD1002D26D1002001213B
:106C30003300009A7A4F53404246101A4A460A439C
:106C40009200BA581D009746009B2C009A468B462E
:106C50005B46022B31D15346FF21002438E0002C43
:106C600017D1042399460023984601339B46AFE78A
:106C7000FF20002D0BD10221DAE7280000F012FEE0
:106C8000431F9D4076235B42181A0021AFE7032182
:106C9000ADE7200000F006FE431F9C4076235B42D8
:106CA0001B1A9846002399469B4691E70C23994668
:106CB000F3339846FC3B9B468AE7032B00D1A5E0C3
:106CC0005546012B00D081E00123002100242B40F8
:106CD0006402C905600ADB070843184303B03CBCE3
:106CE00090469946A246AB46F0BD80240023E403BB
:106CF000FF21EDE7FF210024EAE70123591A1B29B0
:106D000066DD019A134000210024E1E78023DB03C4
:106D10001C4238D01D4251D01C436402640A330027
:106D2000FF21D5E763016C01A3423BD21B26002162
:106D3000013801251F0049005B00002F01DB9C4248
:106D400001D81B1B2943013E002EF3D11C00631EFA
:106D50009C410C4301007F310029CEDD630704D044
:106D60000F232340042B00D00434230103D501005A
:106D70002C4B80311C40FE290DDD0123019AFF219F
:106D800013400024A4E78023DB031C436402640A4D
:106D90003300FF219CE70123019AA401640AC9B2D0
:106DA000134095E71B1B1A260121C2E7009B8B4667
:106DB0009A4600244CE76302E5D500258024E403CD
:106DC0002C436402640A009BFF2181E70195C1E71F
:106DD00023002020CB40411A8C40611E8C411C4373
:106DE000630704D00F232340042B00D00434630135
:106DF00005D50123019A01211340002468E70123EE
:106E0000019AA401640A1340002161E78023DB0397
:106E10001C436402640A5346FF2159E7607A00006C
:106E2000A07A0000FFFFFFF770B5420045024E0256
:106E30004C00C30F6D0A120E760A240EC90F0120F2
:106E4000FF2A06D0FF2C03D0A24201D1B54206D0C2
:106E500070BD002DFCD1FF2CFAD1002EF8D18B4251
:106E600006D00120002AF3D12800451EA841EFE7F3
:106E70000020EDE7F0B5420045024C02C30F480088
:106E80006D0A120E640A000EC90FFF2A1ED0FF28D9
:106E900021D0002A0AD16E426E41F6B200280FD1ED
:106EA000002C0DD10020002D09D005E0002801D1D3
:106EB000002C01D08B4211D0012158420843F0BD73
:106EC000002EF7D0012001390843F8E7002DDED06D
:106ED00002204042F3E7002CDBD0F9E78242EBDCF2
:106EE00004DBA542E8D80020A542E8D20121581EC3
:106EF0000843E4E7F0B542004D024C004602760A32
:106F0000120EC30F6D0A240EC90FFF2A16D0FF2CD4
:106F100018D0002A0AD170427041C0B2002C15D09E
:106F2000002805D0012001390843F0BD002C13D002
:106F3000994214D001205B421843F6E70220002E4C
:106F4000F3D1E4E70220002DEFD1E2E7002DE7D1F5
:106F50000020002EE9D0EDE7002DE9D1EAE7A242BA
:106F600006DCDFDBAE4203D80020AE42DAD3DCE73A
:106F7000012049420843D8E7F8B557464E464546F2
:106F8000DE46E0B54702460088467F0A360EC40F4B
:106F9000002E47D0FF2E24D0FB008027FF041F4384
:106FA000002399469A467F3E43465D025800DB0F18
:106FB0006D0A000E984643D0FF283BD0EB00802599
:106FC0000022ED041D437F383618731C41469B4652
:106FD0004B46614013430F2B64D875489B00C35840
:106FE0009F46002F42D108239946063BFF269A462A
:106FF000DAE74146022A28D0032A00D1CEE0012A4E
:1070000000D0ACE0114000200022CCB24002D205FA
:10701000400AE407104320433CBC90469946A246F0
:10702000AB46F8BD002F15D104239946033B00263B
:107030009A46B9E7FF200222002DC5D00322C3E7FC
:10704000002D19D100200122BEE70124FF220C40AF
:107050000020DBE7380000F025FC7626431F9F4028
:1070600000237642361A99469A469DE70C239946A4
:10707000093BFF269A4697E7280000F013FC431FC0
:107080009D4076235B42181A00229DE78020002451
:10709000C003FF22BAE73D005246ABE73D002100A6
:1070A0005246A7E73B0C9C462A04120C2B0C1400FA
:1070B000604665463F043F0C7C4342435D437B434F
:1070C000270C9B18FF18BA4203D980235B029C4609
:1070D000654424043A04240C121993015C1EA34154
:1070E0003F0C920E7D191A43AD0115432B0104D5B7
:1070F00001235E466A081D40154332007F32002A94
:1071000025DD6B0704D00F232B40042B00D0043562
:107110002B0103D53200274B80321D40FE2A94DC20
:107120000124A801400AD2B20C406FE78020C003BE
:10713000074207D0054205D128434002400A444691
:10714000FF2263E738434002400AFF225EE7012442
:10715000A31A1B2B05DD0C400022002056E75E46DB
:10716000CBE72A002020DA40C31A9D402B005D1E89
:10717000AB4113435A0704D00F221A40042A00D00F
:1071800004335A0104D5012401220C4000203DE7BC
:1071900001249B01580A0C40002237E7802001247B
:1071A000C00328434002400A0C40FF222EE7C0469D
:1071B000E07A0000FFFFFFF741024300C20F490AD7
:1071C0001B0E00207E2B0DDD9D2B0CDC802000048F
:1071D0000143952B0ADC9620C31AD9404842002A65
:1071E00000D108007047034BD018FBE7963B99404D
:1071F000F4E7C046FFFFFF7F70B5002830D0C3170B
:10720000C4185C40C50F200000F04CFB9E231B1AE5
:10721000962B0DDC9622D21A94402A006402640A4E
:10722000DBB26402DB05600AD2071843104370BD6D
:10723000992B19DC9922D21A002A29DD94402200C8
:10724000144C1440510704D00F210A40042A00D0E6
:107250000434620113D4A401640ADBB22A00E0E71B
:10726000002200230024DCE705222100121AD1406D
:10727000B922D21A9440621E94410C43DAE7054BBE
:107280002A001C409F23A4011B1A640ADBB2C8E732
:107290002200D5E7FFFFFFFBF0B557464546DE4627
:1072A0004E46E0B50C0398464E00230B87B007000E
:1072B00092469B46760DCD0F002E6BD06D4B9E42B5
:1072C00035D080245B46420F2404DB0014431C436A
:1072D000C3009946684BA3469C460023002766449A
:1072E000029343461C035A00DB0F5046240B520DF9
:1072F000984600D176E05F4B9A426DD08023410FD3
:107300001B040B435C49E4008C461C43C300002073
:1073100062444146B6186940721C01919446074385
:107320000F2F00D9B0E0554ABF00D25997465B46AF
:107330000343994600D087E000239B460233082789
:107340000293CEE742460192022867D0032800D17B
:107350000EE2012800D062E10023002400229946B9
:1073600001990140CDB2002112030B0D120B1B0538
:107370001343434A240513401C436400ED0764088B
:107380002C434846210007B03CBC90469946A24693
:10739000AB46F0BD034399464FD05B46002B00D16E
:1073A00089E1584600F07EFA03000B3B1C2B00DD00
:1073B0007AE11D22D31A3A0001005C46DA4008390E
:1073C0008C4013008F4023439B46B94600232D4E2B
:1073D0000027361A029384E7534623432AD1002418
:1073E000022096E75346234320D0002C00D157E1DA
:1073F000200000F057FA03000B3B1C2B00DD49E195
:107400001D21CB1A51460200D9405346083A9440F8
:1074100093400C431B4A121A00207AE70125019B76
:10742000144C1D400023002299469CE700240022B2
:1074300001206EE7534603206BE700239B46013390
:107440000427002602934CE7032381460C2702936E
:1074500047E780220023002512039946054C82E766
:107460005C464B4602986FE75C464B460195029896
:107470006AE7C046FF07000001FCFFFF207B000019
:10748000FFFF0F800DFCFFFF4A464946170C1A0C00
:107490001B041B0C08041900000C4143150088460E
:1074A00019007D437943039589462900150045431A
:1074B0004D44029545462D0CAA46029D5544A945CA
:1074C00006D98A46802149028946CA445146039119
:1074D000290C0491414609042D04090C8846290011
:1074E000250C24044144240C059121004143884685
:1074F000210079438A466843414650448146080C3E
:1075000048446F43824503D98021490289464F444C
:10751000010C894639004944029141460F040499FF
:107520003F0C88460004C0198044414604915946E6
:107530000F0C0904090C884659438A463900514307
:10754000894641464A435146090C8B467B43D21833
:107550005A44934203D980235B029B46D944514647
:107560000904090C8A46414661437C43130C12040A
:107570004B445244A1468A463C0041466C434D432D
:1075800051464D440F0C7D19A94503D9802149026C
:1075900088464444049F0399B84641448B4683453A
:1075A000804141428846514608042F04000C3F1890
:1075B0005846029910188946904292414F44BA4663
:1075C000524299469346C244D144CB448F42BF4174
:1075D000C245894199459B41934592417F42494229
:1075E0002D0C52420F435B4213437F19FF185B4639
:1075F0003C19DB0D059A64021C43430213435D1ED4
:10760000AB415A46C00D034352021343E20156D523
:1076100001205A0803401343E207134364085A4801
:10762000604400284DDD5A0709D00F221A40042A71
:1076300005D01A1D9A429B415B42E4181300E201F7
:1076400004D58020514AC00014406044504A904202
:1076500000DDE3E60125DB0862071A436402019BB3
:107660009146220B4405640D1D407CE6802259465C
:107670001203114208D0144206D122431203120B06
:1076800045469946434C6EE65B461A431203120B7D
:10769000404C68E603005446283B9C400023B9E672
:1076A00000F000F92030A6E60300283B9F400023AD
:1076B000BB4699468AE600F0F5F8203074E6B446F9
:1076C000ADE701252A1A382A06DD019B00241D405A
:1076D00000230022994646E61F2A21DC20252000AF
:1076E000AD1A1E00AB40A840D6405D1EAB413043F2
:1076F0001843D440430709D00F230340042B05D07F
:107700000300181D98429B415B42E418230221D5D7
:107710000125019B01241D4000230022994622E6F9
:107720001F2521006D42281AC1400800202A1DD0C3
:107730005F35AA1A944023435C1EA34107250343E7
:107740001D400022002D09D00F2200241A401800ED
:10775000042AD6D1030065076402220BDB082B4301
:1077600001259946019B00241D40FCE50024E2E729
:10777000802201251203224301991203120B0D40AE
:107780009946044CEFE5C046FF030000FFFFFFFEF3
:10779000FE070000FF07000030B5134D0A034B0041
:1077A000120B5B0DC90F0024AB4210DD0F4CA3423E
:1077B0000FDC80240E4D64032243ED1A1F2D0BDDD8
:1077C0000C48C31ADA405442002900D114002000AA
:1077D00030BD094BCC18FAE7084CE840A446634496
:1077E0009A400243EFE7C046FE0300001D0400007C
:1077F0003304000013040000FFFFFF7FEDFBFFFFD9
:107800004100090E4B1C70B5DBB24602750AC40F6D
:10781000012B14DDE0239B006D07360BCB180021F4
:107820000A0D280012051C4D32435B052A405B08F7
:1078300013435B00E4075B082343190070BD002974
:1078400014D1002D1ED0280000F02CF80A281CDCD2
:107850000B232A001B1ADA40030015339D400F4BFF
:1078600012031B1A5B05160B5B0DD8E7002D06D023
:10787000320B802636036D071643094BCFE7084BC2
:107880000026CCE700230026C9E703002A000B3BB3
:107890009A400025E3E7C046FFFF0F808903000000
:1078A000FF0700001C2101231B04984201D3000C98
:1078B00010391B0A984201D3000A08391B09984263
:1078C00001D30009043902A2105C40187047C04679
:1078D0000403020201010101000000000000000099
:1078E000002103E00A4B5B584350043109480A4B1E
:1078F00042189A42F6D3094A02E000231360043288
:10790000074B9A42F9D3FEF7B3FE00F00BF870472D
:107910008C7B000008FEFF1FB8FEFF1FB8FEFF1F94
:107920003C040020A021164B164AC90410B5D150C2
:1079300062B6FAF7B1FCFAF7C3FBFAF724FDFDF7DC
:1079400073FAFDF7D3FDFDF76AFBFAF71FFD0E4C46
:10795000A078FAF71BFCE078FAF782FCFEF7E2FC6D
:10796000FAF736FDFBF720FBFDF726FD2022074B3B
:107970009A60FBF7ADFBFDF79DFBFDF71EFDF8E7F9
:1079800004100000007004400CFEFF1F40F00F4088
:107990008025000040380000004B0000807000008F
:1079A0000096000000E10000002C010000C2010070
:1079B0000084030090D0030020A1070040420F0084
:1079C00050C3000088130000018008080000000078
:1079D00000000000C80000000100000000000000DE
:1079E0000101010001000000000000000000000093
:1079F0000000010000000000000000000000000086
:107A00000101010000000000000000000001000072
:107A1000000000000101010001010001010000005F
:107A20000000000000000000000000000000000056
:107A30000000000000000000000000000000000046
:107A40000000000000000000000001010000000133
:107A50000001000100000000000000000000000024
:107A6000246D0000F46C0000066D0000486C0000FE
:107A7000066D0000EA6C0000066D0000486C000016
:107A8000F46C0000F46C0000EA6C0000486C00002C
:107A9000506C0000506C0000506C00000C6D000039
:107AA000F46C0000F46C0000C86C0000AC6D0000C9
:107AB000C86C0000EA6C0000C86C0000AC6D0000EF
:107AC000F46C0000F46C0000EA6C0000AC6D000087
:107AD000506C0000506C0000506C0000B66D00004F
:107AE000A4700000F46F0000F46F0000F26F00005B
:107AF00096700000967000008C700000F26F00001D
:107B0000967000008C70000096700000F26F00000C
:107B10009C7000009C7000009C7000002C710000A4
:107B2000887400004873000048730000447300002C
:107B30006074000060740000527400004473000020
:107B40006074000052740000607400004473000010
:107B50006874000068740000687400006C760000AF
:107B6000313231305631313200000000F8B5C046B4
:107B7000F8BC08BC9E467047F8B5C046F8BC08BCC7
:047B80009E46704766
:047B840039200000A4
:047B880011200000C8
:107B8C00607B00000102000000000000000000000B
:107B9C0000000000080002000100000000000000CE
:107BAC000000000000000000006CDC0272B67022C5
:107BBC000B4B1A701A7852B2002AFBDA0922DA71CE
:107BCC00020CD2B29A71020AD2B25A718022C0B29D
:107BDC0018711A701A7852B2002AFBDA62B6704722
:107BEC000000024072B67022104B1A701A7852B212
:107BFC00002AFBDA0622DA71020CD2B29A71020A5E
:107C0C00D2B25A71C0B20A0E1871DA720A0CD2B220
:107C1C009A720A0AD2B25A728022C9B219721A70B6
:107C2C001A7852B2002AFBDA62B6704700000240A2
:107C3C008C7B000008FEFF1FB0000000000000005D
:087C4C00000000000000000030
:020000041FFFDC
:04FE000000000000FE
:04000003000078E1A0
:00000001FF
